:060000000A128A11122809
:10000800FE00030EF1000408F2000A08F300831250
:1000180003137F08F4000A128A11E02C0A128A11CD
:10002800822D8B010730831603139F00831203135D
:100038008501831603138501831203138601831632
:1000480003138601803083120313870080308316E0
:1000580003138700043081007D3083120313BC0032
:100068003C08BF00A301A0012030B8000030B9004F
:100078000A30BA000030BB0024300A128A112F253A
:100088000A128A11203083120313B8000030B90015
:100098000A30BA000030BB002E300A128A112F2510
:1000A8000A128A11F81183120313A101781178102A
:1000B800F810A201063081008B160A128A118E25CB
:1000C8000A128A118B170A128A112A240A128A1113
:1000D80083120313B80100300A128A1152250A123A
:1000E8008A11233083120313B8008030B9000A1232
:1000F8008A110A250A128A1183120313B801B80A51
:1001080000300A128A1152250A128A11013083120C
:100118000313B8008030B9000A128A110A250A129E
:100128008A1183120313BE0114303E020318AF284C
:100138008230BD00DD30BC00BC0BA028BD0BA02860
:10014800A528013083120313BC003C08BE071430F5
:100158003E02031C9C28B80100300A128A1152255D
:100168000A128A11013083120313B8008030B900D3
:100178000A128A110A250A128A1183120313B80176
:10018800B80A00300A128A1152250A128A1112304E
:1001980083120313B8008030B9000A128A110A25A5
:1001A8000A128A1183120313BE010A303E02031891
:1001B800F0288230BD00DD30BC00BC0BE128BD0B4F
:1001C800E128E628013083120313BC003C08BE076F
:1001D8000A303E02031CDD28B80100300A128A11D9
:1001E80052250A128A11123083120313B800803084
:1001F800B9000A128A110A250A128A1183120313F6
:10020800B801B80A00300A128A1152250A128A1156
:10021800673083120313B8008030B9000A128A11BC
:100228000A250A128A1183120313BE010A303E02FC
:10023800031831298230BD00DD30BC00BC0B2229F7
:10024800BD0B22292729013083120313BC003C0867
:10025800BE070A303E02031C1E29B80100300A12EC
:100268008A1152250A128A11673083120313B800C3
:100278008030B9000A128A110A250A128A118312DB
:100288000313B801B80A00300A128A1152250A125B
:100298008A11893083120313B8008030B9000A121A
:1002A8008A110A250A128A1183120313BE010A3021
:1002B8003E02031872298230BD00DD30BC00BC0B41
:1002C8006329BD0B63296829013083120313BC001D
:1002D8003C08BE070A303E02031C5F29B801003003
:1002E8000A128A1152250A128A11893083120313BD
:1002F800B8008030B9000A128A110A250A128A1138
:1003080083120313B801B80A00300A128A11522561
:100318000A128A11343083120313B8008030B900EE
:100328000A128A110A250A128A1183120313BE01BE
:100338000A303E020318B3298230BD00DD30BC000C
:10034800BC0BA429BD0BA429A929013083120313CE
:10035800BC003C08BE070A303E02031CA0290A1252
:100368008A11C1230A128A11831203138C1E4D2A83
:100378008C129818C129181DCC29981CC529181247
:100388001816181D4D2A1A08BC003C08A0004D2A52
:100398001A08BC003C08A0002008783A031DDA2996
:1003A800F8157D30BC003C08A2004D2AF81D4D2AE6
:1003B8000A3021020318EC292008BC002108243E39
:1003C80084003C08831380000130BC003C08A1076E
:1003D8000A302102031C4D2A2430BC003C08F500D9
:1003E8000A30F6000030F7002E300A128A117924FC
:1003F8000A128A11760875040319042A7815052A41
:100408007811243083120313BC003C08F5000A302D
:10041800F6000030F7002E300A128A1179240A12E9
:100428008A1176087504031D1B2A78141C2A781073
:10043800243083120313BC003C08F5000A30F60090
:100448000030F7002E300A128A11B5240A128A11D8
:100458000A128A11C1230A128A11F811831203138E
:10046800A101BE010A303E0203184D2A8230BD00A8
:10047800DD30BC00BC0B3E2ABD0B3E2A432A0130AE
:1004880083120313BC003C08BE070A303E02031C5B
:100498003A2AF81D6F2AA208031D6F2A78117810CE
:1004A800F814F811A101BE010A303E0203186F2AA0
:1004B8008230BD00DD30BC00BC0B602ABD0B602A59
:1004C800652A013083120313BC003C08BE070A30BA
:1004D8003E02031C5C2A781D752A831203138715B4
:1004E800782A831203138711781C7E2A8312031338
:1004F8000715812A831203130711F81C872A831210
:0E05080003138714B829831203138710B82930
:10060000FF1B0A2B83137F1883170008840A031922
:10061000FF0A080003308A000408840A82070034B5
:1006200020342034203420342034203452344634D2
:1006300049344434203420342034203420342034CD
:100640000034203420342034203420342034463404
:100650005234493447342034203420342034203478
:1006600020340034203420342034203443347A348D
:10067000793474346E3469346B342034203420344B
:1006800020342034003420342034203431343934C0
:10069000373434342D34323430343134343420343B
:1006A00020342034203400342034203442344C347C
:1006B0004134443420344B344C34553443345A346C
:1006C0004134203420342034003420342034203489
:1006D0004E344F345734593420344B344C34553421
:1006E00043345A342034203420340034203420342D
:1006F000283443342934203465344B3461346D3428
:1007000053346F34663474342034203400344F341E
:1007100043345A3445344B3455344A344534203408
:100720004B344C34553443345A344134203400343F
:100730002034623479342034523461346634613484
:100740006C34203453347A3475346C34633420344C
:10075000003450344F34573454344F3452345A34B4
:100760004F344E34593420344B344C3455344334A4
:100770005A3400344B344C34553443345A343A34BC
:1007800000340A128A11B3250A128A118312031344
:10079000B80100300A128A1152250A128A11AB30B0
:1007A00083120313B8008030B9000A128A110A2597
:1007B0000A128A112E3083120313B8000030B900D8
:1007C0000A128A110A250A128A1183120313B80128
:1007D000B80A00300A128A1152250A128A11781DAD
:1007E000FC2B563083120313B8008030B9000A1274
:1007F0008A110A250A128A11781C092C9A30831250
:100800000313B8008030B9000A128A110A250A12AF
:100810008A11F81C162C453083120313B80080305F
:10082000B9000A128A110A250A128A11781D78184D
:10083000262CF818262C783083120313B800803049
:10084000B9000A128A110A250A128A110A128A119B
:10085000B7250800413083120313BB00EE30BA0005
:10086000BA0B302CBB0B302C000083120313071281
:100870000713871230308600071707130D30BB00AF
:10088000FB30BA00BA0B422CBB0B422C472C303049
:10089000831203138600071707134230BA00BA0BFE
:1008A0004F2C000030308312031386000717071304
:1008B0004230BA00BA0B5A2C000038300A128A11A2
:1008C000A2250A128A1108300A128A11A2250A12D8
:1008D0008A110A128A1164250A128A1106300A1234
:1008E0008A11A2250A128A110C300A128A11A22535
:1008F000080083120313BA000130F6020030031C13
:10090000F703F702FF307706031D882CFF307606C9
:100910000319B22C7508840083130008B8003A0844
:100920008400000838060319A92C75088400000803
:10093000B800B901B809B909B80A0319B90A3A08DF
:10094000840000083807F50039080318390AF60052
:1009500008000130B8003808BA070130B80038087C
:10096000F5077C2CF501F601080083120313B9008A
:100970007508B8003808BB003908B8003808BA0054
:100980000130F6020030031CF703F702FF30770650
:10099000031DCC2CFF307606031908003B088400A9
:1009A00083130008B8003A0884003808800001303A
:1009B000B8003808BB070130B8003808BA07C02CA7
:1009C0000B1DFF2C0B11063081000130BF02BF0848
:1009D000031DF22C7D30F0007008BF000430F000E1
:1009E0007008A30023080319F92C0130A30207148F
:1009F000FA2C071022080319FF2C0130A2027408F8
:100A0000FF0073088A0072088400710E8300FE0ED6
:100A10007E0E0900831203133908FF003808840092
:100A20000A128A1100230A128A11003803190800D9
:100A3000831203133908FF00380884000A128A1150
:100A400000230A128A110A128A1199250A128A11A0
:100A5000013083120313B8070318B90A0A2DF600F0
:100A60007608F5007508F700013083120313BA0207
:100A70000030031CBB03BB02FF303B06031D422DAD
:100A8000FF303A0603190800831203133808F500F3
:100A9000770884007508831380000130F50075081D
:100AA000F707342D83120313BA003808B900063053
:100AB0000310B90DFF3E031D582D3A083907803E3B
:100AC0000A128A11A225080001300A128A11A225F1
:100AD0000A128A11073083120313B9007D30B8005F
:100AE000B80B702DB90B702D0800F6007608831234
:100AF00003138600071707134230F500F50B7E2D10
:100B000000000800F80183132030840038300A12F6
:100B10008A11AB2583010A128A1115288316031343
:100B20001815193099001812831203131813181688
:100B30000800F70083120313071677080A128A11B8
:100B400075250800F70083120313071277080A12AD
:100B50008A117525080064008001840A04060319BF
:100B600000340406AC2D831203139813080083127B
:060B7000031398170800B2
:02400E0071FF40
:00000001FF
